:1000000012C0189518951895189518951895189563
:1000100018952DC018951895189518951895189538
:100020001895189518958FE58DBFC0E4E8E34E2E1E
:1000300084E08EBFD4E0F4E05F2EEEEFF3E0A0E6C4
:10004000B0E088278D933197E9F784B7082E877F32
:1000500084BF8FE181BD87E081BD662483B7816065
:1000600083BF89B7816089BF81E682BF2DC00F93AE
:100070008F938FB78F93AF93BF939F93A0E6B0E01A
:100080008D919C9101969C938E93002781309007CF
:1000900011F4949A0FC0903041F0803D07E0900732
:1000A00048F000270D930C9305C012969D91891777
:1000B00008F0949881E682BF9F91BF91AF918F9194
:1000C0008FBF8F910F911895789487E886B980E05B
:1000D00087B9379A8D988A9AA498A598E1E0F0E0BC
:1000E000A5E6B0E092E08CD1E2E0F0E0A7E6B0E077
:1000F00092E086D1A5E6B0E00D911C910F3F5FEF35
:10010000150709F006C084E690E0A5E6B0E08D93FF
:100110009C93A7E6B0E00D911C910F3F5FEF150790
:1001200009F006C084E690E0A7E6B0E08D939C93CA
:100130008091650080936200929A0027A0E3B0E06E
:100140008C9185FB0EF401E040E0041709F010C02B
:10015000E2E0F0E015D192980027A0E3B0E08C91A6
:1001600085FB0EF401E040E0041709F001C04BD01C
:10017000929A07B1007F056007B91FD1A3E6B0E0EE
:100180008D939C93A3E6B0E00D911C9144E050E068
:100190000AD1A3E6B0E00D931C93A3E6B0E00D9165
:1001A0001C9100315EE0150710F009F001C006C097
:1001B00080E19EE0A3E6B0E08D939C93A3E6B0E0DF
:1001C0000D911C910A3050E0150708F006C08AE036
:1001D00090E0A3E6B0E08D939C93EAE0F0E0D0D00D
:1001E0008091670080936200E2E0F0E0C9D08091E6
:1001F000650080936200A3E6B0E0ED91FC91C0D071
:10020000EFCFF894FFCFE1E0F0E0BAD0929A07B1D7
:10021000007F046007B9D1D0A5E6B0E08D939C9330
:10022000A5E6B0E00D911C914AE050E08FD0A5E624
:10023000B0E04D935C93A5E6B0E00D911C914DE2CA
:1002400050E0040F151FA5E6B0E00D931C938091BC
:100250006500809362000027A0E3B0E08C9185FBED
:100260000EF401E040E0041709F0D1CFE1E0F0E046
:10027000A5E6B0E092E07BE7B2D09298E1E0F0E052
:100280007FD0929A07B1007F046007B996D0A7E6A5
:10029000B0E08D939C93A7E6B0E00D911C914AE0ED
:1002A00050E054D0A7E6B0E04D935C93A7E6B0E0F1
:1002B0000D911C914DE250E0040F151FA7E6B0E030
:1002C0000D931C9380916700809362000027A0E348
:1002D000B0E08C9185FB0EF401E040E0041709F0DA
:1002E000D1CFE2E0F0E0A7E6B0E092E07BE777D0A4
:1002F0009298E1E0F0E044D0809165008093620044
:10030000089508D050D000FC10D0089503D01ED01E
:1003100001F8F9CF0024E89457FF02C009D068948F
:1003200000F80BD010F80124089502D009D00895E8
:10033000509540954F5F5F4F0895E89417FF0895DB
:10034000009510950F5F1F4F68940895352F242F47
:10035000E894452B11F468940895512F402F0027FD
:10036000112780E1440F551F001F111F021B130BA3
:10037000416018F4020F131F4E7F8A9599F7089574
:1003800008950895689462F80895E89462F80895CD
:10039000EF93FF93EE27E82BE92B11F0E0EAFFE063
:1003A000FF91EF9108950F92B801469F8001479FFA
:1003B000100D569F100D0F900895369A3699FECF66
:1003C000369A3699FECF84B195B10895E199FECF62
:1003D000EEBBFFBB3196089591E001C092E07B3700
:1003E00051F47FB7F894F2DF8D918DBBE29AE19AD8
:1003F0009A95C9F77FBF7727089591E001C092E0F1
:0E040000E5DFE09A8DB38D939A95D1F70895BC
:00000001FF
